:0A0000007D28000000000000B52874
:100020002D2AE928ED28FD28032909290F29080090
:10003000E728E728E728E72808000800F128F5283E
:10004000E528E528E528E528E528E528E528E3284A
:10005000152A072AFA29EC2908000800E528E528CE
:10006000242AE928ED28F928FF2805290B29E52865
:10007000E528E528E528080008000800F128F5280B
:10008000342A352A392A452A492A4D2A512A552AFD
:10009000592A5F2A652A6B2A080008003D2A412A4E
:1000A00077341434D334D534B434E534E7345434A9
:1000B000F734F534F634A73463349734E334E23458
:1000C000E7348134B634B534D13475347734A1345F
:1000D000F734F534F3345734663497347634723465
:1000E000A6000F308F050F0864008A010310260751
:1000F000820083018B01792800008316003085007F
:10010000FE3086008730810083128B018B168B179F
:10011000850186010830A5008F01E7220319A42874
:100120001130960038309500013098000030990069
:1001300001309A0000309B0001309C0001309D008E
:1001400001309E0001309F0032214B21612111219D
:10015000342332227622A1220530CA009C230510C6
:100160000530CA009C230514AC28640094000308E1
:1001700093002808A90000300F040319C128A5180E
:10018000A9017622A50BD5280830A500861CE028F9
:10019000061DDD28861DDA28D52832214B21612154
:1001A0001121342332227622A1221308830014085D
:1001B0000B11090030307020CD2820307020CD2860
:1001C00010307020CD288F0108008F0A08008F039F
:1001D000080098090130980508009909013099052F
:1001E00008009A0901309A0508009B0901309B0517
:1001F00008009C0A03309C0508009C03FA289D0A0D
:1002000007309D0508009D0300299E0A07309E05C2
:1002100008009E0306299F0A07309F0508009F03D8
:100220000C291608A1001508A2000310A20DA10DAB
:100230002113191821171F08A300A30EA3170310D9
:100240001E0DA3041D08A4000310A40DA40D1C087A
:10025000A4040310A40DA40D241118182415A4102F
:100260002410080064009613161396121608031043
:100270000D3C0318412916080310183C031C46299D
:1002800008000E309600B830950008000E30960039
:10029000B83095000800640066211508C4001608EF
:1002A000C3000310C40DC30DC40DC30D25300310CE
:1002B000C302C401922133089700970E31089704B6
:1002C0000800640066217721922108006400C301C0
:1002D000C401C501B101B301B501B701B901BB0149
:1002E000B001B201B401B601B801BA01080064005E
:1002F0001508AF001608AE006400083090007D308D
:10030000C00003106400C00C031C8C292F08C40714
:100310002E0803182E0FC507C50CC40CC30C900B78
:10032000822908000130B0004308D1214408D121BE
:100330004508D12108000630900030308400AC011F
:1003400064002C08AD00AC01AA21840A840A900B39
:10035000A02908000310800D2D18800AC32906303B
:10036000900030308400AC0164002C08AD00AC017A
:10037000BD21840A900BB42908000008840A2D18B6
:10038000800A03108007001ACC29801D080000197C
:10039000CC298018CC2908000630800700122C14C4
:1003A0000800C20008308C004218AF219B21C20C0B
:1003B0008C0BD429080003102E0895070318AF0AE8
:1003C00003102F089607080003102E089502031C3F
:1003D00096032F089602080003103508083C0319FD
:1003E000F6290310950A0318960A08000730AE0094
:1003F000AF01E42937080310093C0319032A083028
:10040000AE00AF01DB294830AE00AF01E429390866
:100410000310093C0319102A5030AE00AF01DB294C
:10042000D030AE000230AF00E4293B080310093C95
:1004300003191F2A2030AE000330AF00DB29203023
:10044000AE001C30AF00E4294030AE00AF01DB212C
:10045000C03015053838950008004030AE00AF01B7
:10046000E421282A403070288D2A6230A80018081C
:10047000732AF630A8001908732A9730A8001A08C2
:10048000732A8730A8001B08732A6330A8001C0851
:10049000712AB630A8001D08712AF230A8001E0883
:1004A000712AE230A8001F08712A0730A8003B0813
:1004B000732A3B089100910E390811048E2A3908DD
:1004C0009100910E370811048E2A37089100910E81
:1004D000350811048E2A35089100910E3308110455
:1004E0008E2A0310013E9D22A700080064002908FF
:1004F0008E00802227088E00802206140610080035
:1005000008308D008E09640085118E1B8515051538
:1005100005118E0D8D0B832A08001708920091009B
:100520009D22A700120E91009722A80008009100BA
:100530005030A60011080F39742891006030A600D1
:100540009A2A8B01A001890116080310A0078800D0
:100550002623890A15080310A00788002623890A84
:1005600018080310A00788002623890A1908031019
:10057000A00788002623890A1A080310A00788000C
:100580002623890A1B080310A00788002623890A4E
:100590001C080310A00788002623890A1D080310E1
:1005A000A00788002623890A1E080310A0078800D8
:1005B0002623890A1F080310A00788002623890A1A
:1005C0002008880026238B018B168B170800A001BA
:1005D00089011F2396000310A007890A1F23950095
:1005E0000310A007890A1F2398000310A007890A97
:1005F0001F2399000310A007890A1F239A000310E4
:10060000A007890A1F239B000310A007890A1F2344
:100610009C000310A007890A1F239D000310A00758
:10062000890A1F239E000310A007890A1F239F0029
:100630000310A007890A1F2303102002080064008A
:10064000831608148312000008080800640083164B
:10065000081555308900AA30890088146400081EE6
:100660002E2B08128312080064007623CA30C700BC
:100670005F2370232108C7005F2370232208C7006F
:100680005F2370232308C7005F2370232408C7005B
:100690005F2370237C230800C8010830C600842330
:1006A0008F23061E542B572B0310C80D5B2B0310F2
:1006B000C80DC80A5B2B9423C60B502B08000830CA
:1006C000C6000310C70D031C662B6A2B89238123E8
:1006D00084236D2B842381236D2BC60B612B080093
:1006E0008423812308008923812308009423842301
:1006F0008F23892394230800942389238F23842321
:1007000008008F23942308008316061683129A2369
:10071000080006128316061283129A230800831615
:10072000861683129A230800861283168612831275
:100730009A2308000530CA006400CA0B9C2B0800ED
:10074000FA30C9006E30CA006400000000000000EA
:0E07500000000000CA0BA42BC90BA22B08004E
:00000001FF
